:0200000038289E
:080008000B1915280B180E2836
:100010008B180B2809008B108D1509000608F03984
:10002000F03A031D8D150B1009000B110C1C1C2838
:1000300005181C2805141D2805108C1E28288C1254
:10004000101E2628910B26281015101200002928B2
:100050008C160E1E2C288F0B09002E2864308F0062
:100060001A1E36289B0B36281A151A120000090092
:100070008130840001308000810185018601853056
:1000800084001A30800086308400F7308000803091
:100090008C0000308D00143092003C3093001430FE
:1000A0009400A001831D5E281E3095005A309600F2
:1000B0001E309700FF30A400061EDD2286110C10B2
:1000C0008B018B168B178E0164308F000E1606087D
:1000D000F039F03A031D6728861876280619762825
:1000E0002C226130082233228D147A280D1B9F2286
:1000F0000D13B4222621060C033982072329002977
:10010000DD2890283D228C197A288B130B168B1230
:100110008B158B1363008B018B168B17A0017A282C
:100120000C1286080608F039F03A031982288C1D53
:10013000A9280D1FA3288C1183308D052C22623035
:1001400008223322D7280D172C2278300822332298
:10015000D7289001643091001016101DAD28060EAE
:100160000F3982070028C828CC28C428C828C828E6
:10017000CA28D428D628C228C628D228C828D028D9
:10018000CE28D728A521D7286C21D728CF21D7283A
:100190002722D7289321D7289F22D728FD22D72886
:1001A0000923D7281323D7287922D728BB2206086A
:1001B000F039F03A031DD7288228A00FE0288728BD
:1001C00086150C140C160C139001120891001016D1
:1001D0008C18ED280310A10DEF280314A10D061DA6
:1001E0000C17101DEF2886110C10900114089100B7
:1001F0001016061D0C17101DF9280C1B23297A2830
:10020000A00F0329872886150C140C120C139001DB
:100210001308910010168C1810290314A10D12292F
:100220000310A10D861C0C17101D122986110C102D
:100230009001140891001016861C0C17101D1C2923
:100240000C1B23297A280C1EDD2800290D180134E7
:100250008B12853084001A30800005080238E73997
:100260008500813084002830800085308400801132
:10027000FF309800980B3A29801598018101801071
:10028000980A011C40291A308000180893001808A9
:100290009D0003309F00D8211D08920094008D1C02
:1002A00057291308960012089500140897008C1C13
:1002B0005F291308980012089300180892008130F3
:1002C0008400013080008101853084008C1F00147F
:1002D0008C1B00108B1600349001C8309100101652
:1002E000101D70299A01C8309B001A1685308400B1
:1002F00000107D3008228615861C9029061D902945
:10030000061E9029861E9029061F9029861F902977
:100310001A198B297C298630840080150030082228
:100320008611332200342C227230082261300822D8
:1003300033221308980012089300180892008C18B2
:10034000A3298C1400348C1000348D1CB2298D101C
:100350002C22613008229A0105309B001A161A1DC2
:10036000AF2900280D1CBB290D1026210C190034C3
:100370002C227A30292A0D141608930015089200B1
:10038000170894008C1CCA291308980012089300BF
:10039000180892000C1900342C227430292A8C1B66
:1003A000D3298C17D4298C132C227B30292A003492
:1003B0009E0108309C001D0D9E0D1F089E02031813
:1003C000E3299E0703109D0D9C0BDB290034861545
:1003D0000C140C169001120891001016101DEE2935
:1003E00086110C100122003486150C140C12900199
:1003F000130891001016101DFB2986110C10012204
:1004000000349001140891001016101D052A0034C4
:1004100098009900FF3A0319013407309C00980DA9
:100420009C0B132A0134980D0318102A8C18980974
:10043000980D031C1D2AF4211E2AE7219C0B182A63
:100440000122991F003401220122012200342C22B2
:100450000030082233220034863084008015853035
:1004600084000010003486308400801185308400C0
:100470008C1F00148C1B001000348C1D0034FE30C7
:100480002102031900348D1E602A23088400A11361
:10049000210880000D1F502A84038017840A0D1341
:1004A000840AFF308000FE30A100A001A30A4F3073
:1004B0002302031D00348C118D1262300822013496
:1004C000A1132108C6220D1B6F22A30AFF30C622EA
:1004D000FE30A100A0010D1222082302592A0D139B
:1004E0000D1A0034A303D72288170808C622A30ACE
:1004F00000349A010A309B001A161A19822A861BA8
:100500008B2A7D2A8C158D162430A300FE30A10085
:100510002C224130292A00008D112430840000084B
:100520000822013C03199D2A8D199D2A0608F639D7
:10053000F63A031D9D2A840A8F2A000000342C22DB
:1005400062300822403008227730082273300822B7
:10055000E4300822613008224F300822153008228A
:1005600047300822332200342C22583008224330EE
:100570000822332200342C228D1BC12A8D176830AB
:10058000C32A8D137A3008223322003488002308CE
:1005900089008B1383160812081555308900AA307C
:1005A00089008814081ED22A83128B17003423086E
:1005B000890083160814831200343D30A3000030F4
:1005C000C6220030A3004F30C622A30A4730C622FD
:1005D000A30AFF30C6223E30A3001F30C6221F30C0
:1005E000A300FF30C6223F30A3003030C622303097
:1005F000A300FF30C6220D1700343D30A300D722E0
:100600000808A3001E308D1B3C30A2004F30A10013
:100610001C2B3E30A300D7220808A3002F30A200D5
:100620004730A1001C2B3F30A300D7220808A300AD
:100630003C30A2004330A1009A010A309B001A16F8
:100640001A19282B0608F039F03A03193E2B202BF3
:100650008C158630840080158530840000102108B8
:100660000822863084008011853084008C1F00149D
:100670008C1B0010FE30A1000D1600348D110D16DC
:100680000C15A201D722523008020319592B0D1262
:1006900008080822013C0319552B0B168B158D19E0
:1006A000552BA30AA20A2621422B0B128B110C11E7
:1006B0000034A303D722A30A881B622B0D1A622BD6
:1006C0005230492BA30AA20AD7220D1AA72B683051
:1006D0000802031DA72BA30AA20AD7225F30080233
:1006E0000319A42B4F30080203198F2B473008023F
:1006F0000319912B433008020319932B4030080251
:100700000319952B5C3008020319972B64300802FB
:100710000319992B7B30080203199B2BFD2B0A3000
:100720009D2B14309D2B1E309D2B32309D2B503035
:100730009D2B78309D2BFA309D2B9A019B001A1629
:100740008D19552B1A1DA02B2208A3023E2B0D122A
:100750006A3088130802031DB62B8B228D19552B86
:100760008B168B152322A20AA30A422B7D308813F5
:100770000802031DE12BA30AA20AD72240308813E6
:1007800008020319CC2B4F3008020319CE2B473037
:1007900008020319D02BFD2B3230D22B6430D22B20
:1007A000C830D22B9A019B001A168D19DE2B8615A4
:1007B0000C141A1DD52B86110C10B02B86110C10A1
:1007C000552B7B300802031DE72B0515B02B793024
:1007D0000802031DED2B0511B02B7A300802031D12
:1007E000F72B051DF52B0511B02B0515B02B61302E
:0E07F0000802031DFD2BB221B02B2722552B32
:00000001FF
